:020000040000FA
:10000000031E080086015F308C000D3084008001E3
:10001000840A8C0B07282C282120840007398406A9
:100020000310840C840C840C041A841704128A01B3
:10003000820701340234043408341034203440344C
:10004000803407398A018207303431343234333412
:100050003434353436343734FF30A2008630F22061
:100060007F30A2008130F2200330A2008830F220DD
:100070001030A2008530F2209A010A30A20005302B
:10008000F2200130A3002C30F7200030A200053010
:10009000F2200630EF208C00FF3047210C080D21A4
:1000A0002208980016084721FF303221031D6628D8
:1000B0001608472101301121220896001608472111
:1000C000FF303721031D6828AA2068289601B42034
:1000D000D2204928962018089A006430F620A020E3
:1000E0001A088C0060304A21472100303221031D5C
:1000F0007B28B4207C28AA201A08472101300D2132
:1001000022089A001A08472100302D21031D6D286E
:10011000B420BE200130A3002C30F7209601C82067
:100120000330A300E830F72049282C288C01053043
:10013000EF208C008C150C08A2000530F22052290B
:100140008C010530EF208C008C110C08A2000530CA
:10015000F22052298C010530EF208C008C140C0801
:10016000A2000530F22052298C010530EF208C00CE
:100170008C100C08A2000530F22052298C010530A9
:10018000EF208C000C150C08A2000530F22052293B
:100190008C010530EF208C000C110C08A2000530FA
:1001A000F22052298C010530EF208C0064304A2166
:1001B000472101303221031DEB280230F6208C014B
:1001C0000530EF208C0064304A2147210130322174
:1001D000031DEB286A28522907300421EC288400EB
:1001E000000852298400220880005229A301A2009D
:1001F0001F2164002308220403190800F730FF3E82
:10020000031DFF282121F9288316F83881050F39AD
:10021000810463000F3081045229A501A400252127
:100220001329A501A4002230840024088007250892
:10023000840F00000318013E031C80075229A30904
:10024000A209A20A0319A30A08002A21A40A031971
:10025000A50A5229A509A4095229A501A4003C21F7
:1002600001395229A501A4003C2102395229A501D6
:10027000A4003C210439522925082302031D4429E6
:100280002408220203190234031C04340134A3019C
:10029000A20052290D20A9000005841B290603197C
:1002A00000340134831264000800FF3FFF3FFF3F2A
:1002B000FF3FFF3FFF3FFF3FFF3FFF3FFF3FFF3F4E
:1002C000FF3FFF3FFF3FFF3FFF3FFF3FFF3FFF3F3E
:1002D000FF3FFF3FFF3FFF3FFF3FFF3FFF3FFF3F2E
:1002E000FF3FFF3FFF3FFF3FFF3FFF3FFF3FFF3F1E
:00000001FF
